:020000040000FA
:020000000628D0
:020008000900ED
:04000C00203084001C
:100010008001840A60300402031C08282A16AB16EB
:10002000FF30A1000130C2000130C300201483164C
:10003000850185158312850107309900C03083162C
:1000400081008312313090008E018F0100308B00CF
:10005000003083168C008312831631309B001C14F1
:100060001A088312A30020302302031C3828A3019E
:1000700064000000A20B5228851943280A30A1070A
:1000800003184A285228201852280A30A102031CBB
:100090004E2852282010FF30A10052282014A10120
:1000A000952052288F08031938288F012308503EC5
:1000B000A6005023D0008A012308783EA6005023D2
:1000C000D1008A012308A03EA6005023D2008A0155
:1000D0002308C83EA6005023D3008A01501BE0200D
:1000E000501A1C21D01A0121D0193521501948214C
:1000F000D11BB521511B0122D11ACD21D21B452282
:10010000D01BC120D018BE21511A5B21D1196D21FD
:1001100051197F21D11891215118A321521B672217
:10012000D21A9222521AD1223828A30A203023024E
:100130000318A301AA012A16AB01AB16A401A5015D
:10014000B001B101B201B301B401B501B601B7010B
:10015000B801B901BA010130C2000130C3008B13EC
:10016000230883161C159A0031309B0055309D00E2
:10017000AA309D009C149C18BB281C1183128B175D
:100180000800B00A0A303002031C0800851205126C
:1001900005111E30B118643031198C303002031C47
:1001A00008000310B10DB1193114B108031931144D
:1001B00031188516B118051631190515B00108005A
:1001C000521CE6282B1885122B180800B00A0A309A
:1001D0003002031C0800B11C8512B1180512FA3058
:1001E000311C2D303002031C0800B10A521DB11021
:1001F0000130D31FB100B11C8516B1180516B0012E
:100200000800B40A0A303402031C0800B51C0511AA
:10021000B5188510F630351C32303402031C080046
:10022000B50AD21CB5100130D31EB500B51C05159A
:10023000B5188514B4010800521C22292B18051288
:100240002B180800B20A0A303202031C08000512FB
:10025000FF30331C37303202031C0800B30A013070
:10026000531FB3000516B2010800B60A0A30360261
:10027000031C08008510F030381C1E303602031CA9
:100280000800B80A0130D31EB8008514B601080072
:10029000B90A0A303902031C08000510F3303A1C71
:1002A00028303902031C0800BA0A0130D31EBA00F4
:1002B0000514B9010800B00A1430311C4630300270
:1002C000031C080085126730311C73303002031C98
:1002D0000800B10A8516B0010800B20A1430331CB8
:1002E00046303202031C080005126630331C72309F
:1002F0003202031C0800B30A0516B2010800B40A52
:100300001430351C46303402031C080005116230DD
:10031000351C6C303402031C0800B50A0515B40105
:100320000800B60A1430381C46303602031C080098
:1003300085106730381C71303602031C0800B80A7B
:100340008514B6010800B90A14303A1C4630390247
:10035000031C0800051064303A1C6E303902031C7F
:100360000800BA0A0514B90108003608B60B0800DF
:100370000508023A8500C830B60008003608B60BFA
:100380000800B70A371C08000508023A8500051066
:10039000851C0514A030B6000800A50FD6291E3014
:1003A000A5000310AA0DAA1AAA15AA122508A400CE
:1003B0000130AA19A40268302A050319E129851021
:1003C00005152A1324080E020318EC2914302A05F7
:1003D0000319EC29851405118F08031D080064001A
:1003E00024080E02031CEC2914302A050319FA29EB
:1003F0008510051528302A050319002A85140511D2
:100400000800521C162AAA302B05031D162AC20BFF
:10041000212AC30B212A2B1804302B1902302B1A46
:1004200002302B1B7830C300FF30A500A50F212A16
:100430001E30A5000310AB0D03182B140310521C23
:10044000AB0D2508A4000130AB19A402AB1BA4021C
:10045000CC302B05031D051024080E020318342A86
:1004600033302B05031D05148F08031D080064009D
:1004700024080E02031C342A33302B05031D0510FB
:10048000CC302B05031D05140800B00A0A303002D9
:10049000031C0800851205120511851005107D301A
:1004A000311C53303002031C0800B10A0330B1057F
:1004B000B1080319851603190516B1180515B118E9
:1004C00085143118652AB1180514B0010800B00A66
:1004D0001E30B1193230311A1E303002031C0800B0
:1004E000851205120511023031192830B119643016
:1004F000311A96303002031C08000310B10DB11AF6
:100500003114B1080319311419303105031D851652
:100510001A303105031D05161C303105031D051564
:10052000B0010800B00A1E30B11A3230311B1E3043
:100530003002031C080085120512051185100510F4
:100540000230311A2830B11A6430311B9630300233
:10055000031C08000310B10DB11B3114B1080319BD
:1005600031146130D21941303105031D85166230D6
:10057000D21942303105031D05166430D2194430BA
:100580003105031D05156830D21948303105031DAA
:1005900085147030D21950303105031D0514B00197
:1005A00008000130C00203180800E130C00001302B
:1005B000C102031808000130C100B00A0130300246
:1005C0000319182B16303002031985121830300227
:1005D000031905121A303002031905111C303002BC
:1005E000031985101E30300203193B145A303002B3
:1005F00003193B105B303002031905145F303002E1
:10060000031985146430300203190515693030026E
:10061000031905166E30300203198516E6303002D4
:100620000319B0013B1C08000508013A85000800C9
:0C06300085160516051585140514080034
:1006A00003308A000530260782007C3474347834A5
:1006B00070347C347434783470345434503444346A
:1006C00040346C346434683460346434603460348E
:1006D00000348C3482347C3474347034003400340C
:1006E0000C340034003400347034003400340034EE
:1006F000003400340034003400340034803440349A
:10070000C034003480344034C034203421342034A8
:100710002134003480344034C03400340134403457
:100720000034003400340034803403341F349D34EA
:100730000034003400340034C03400340034003459
:100740000034003400340034003400340034003409
:1007500000340034003400340034003400340434F5
:1007600004340434043404340434063406340634C3
:10077000803406340634003400340034003400344D
:10078000423420342834103401340034003400342E
:1007900000340034003400340034003400340034B9
:1007A0000034E034E034E034E034E034E034E03489
:1007B000E034E034E034E034E034E034E034E03499
:1007C0000034E034E0348034803480340034003449
:1007D0002034003400340034203400340034003439
:0A07E000003400340034003400340B
:084000000000010001000800AE
:02400E00CC01E3
:00000001FF
